:10000000A5286820A0000408A2000800A000652020
:100010008413C8309200003093008A208C0A910A21
:100020008E018F0100082005920064000008200561
:10003000930012061305200603198E0A03198F0A6E
:100040001308920090030319910303198C0B1528D0
:100050000E08A028920022088400093093000310A3
:100060003620920C930B30280314362884139F1DDE
:100070004528000820041F1D200680008417000862
:100080002004031C20068000502800082004031CC4
:1000900020061F192006800084172009800550289B
:1000A0001F0D06398C0059208D008C0A5920000044
:1000B0007B2800308A000C08820701349634033410
:1000C000363400345D340C34FA3484178004A028AC
:1000D0009400063094190530840000308A0014081A
:1000E00007398207013402340434083410342034D0
:1000F000403480348D01FB3E8C008D09FF30031CA1
:1001000084288C07031881288C0764008D0F8128B0
:1001100000000800103094008D018C01930C920CAB
:10012000031C98280E088C070F0803180F0F8D0763
:100130008D0C8C0C910C900C940B8E281008A02820
:1001400083130313831264000800E8308E00033029
:100150008F000630840001300620A4000F08A5009F
:100160000130012006309F0024082A2025082A207B
:06017000A5286300B92878
:02400E00FD3F74
:00000001FF
